:100000000C9462000C948A000C948A000C948A0070
:100010000C948A000C948A000C948A000C948A0038
:100020000C948A000C948A000C948A000C948A0028
:100030000C948A000C948A000C948A000C948A0018
:100040000C94CB010C948A000C943A030C94880312
:100050000C948A000C948A000C948A000C948A00F8
:100060000C948A000C948A000000000024002700F1
:100070002A0000000000250028002B0000000000DE
:1000800023002600290004040404040404040202DA
:100090000202020203030303030301020408102007
:1000A0004080010204081020010204081020000012
:1000B0000007000201000003040600000000000029
:1000C0000000F40411241FBECFEFD8E0DEBFCDBF87
:1000D00011E0A0E0B1E0ECEBFCE002C005900D9275
:1000E000A431B107D9F711E0A4E1B1E001C01D923C
:1000F000A73CB107E1F710E0C4ECD0E004C02297C0
:10010000FE010E942106C23CD107C9F70E944A05A0
:100110000C945C060C940000A0E0B0E0E2E9F0E092
:100120000C942D06EC01A880B980CA80DB80A11454
:10013000B104C104D10441F484E2A82E89EDB82EA3
:100140008BE5C82E87E0D82EC601B5012DE133EF2F
:1001500041E050E00E94040627EA31E440E050E02C
:100160000E94C3057B018C01C601B5012DE133EF6F
:1001700041E050E00E940406CA01B9012CEE34EFC0
:100180004FEF5FEF0E94C3056E0D7F1D801F911F13
:1001900097FF04C061507040804090486883798325
:1001A0008A839B839B01AC015F77B901CA01CDB7FC
:1001B000DEB7EAE00C9449060E948C00089580E0C6
:1001C00091E00E948C0008956093000170930101FA
:1001D000809302019093030108955F926F927F9242
:1001E0008F929F92AF92BF92CF92DF92EF92FF9247
:1001F0000F931F938EE00E94E602682E8FE00E940C
:10020000E602A82E80E10E94E602E82E81E10E942B
:10021000E602082F82E10E94E602582E83E10E9446
:10022000E602882E86E00E94E602C82E87E00E9441
:10023000E602112707FD1095000F111FFF24E7FCB0
:10024000F0940E0D1F1D000F111FBB24A7FCB094CE
:100250000A0D1B1D000F111F772467FC7094060DFB
:10026000171D000F111F992787FD9095080F191F63
:10027000000F111FDD24C7FCD0940C0D1D1D000FB5
:10028000111F992487FC9094080D191D000F111F50
:10029000852D800F1F910F91FF90EF90DF90CF90F1
:1002A000BF90AF909F908F907F906F905F900895D8
:1002B0000F931F930E94ED00682F85EA91E00E9442
:1002C000B4048DE00E94E602019719F560E070E049
:1002D00080E090E024E030E040E050E00E94A5059E
:1002E000062F10E00FC060E070E080E090E02FEF9C
:1002F00030E040E050E00E94A50585EA91E00E94D0
:10030000B4041F5F10177CF385EA91E06DE00E9452
:10031000B40468EE73E080E090E00E9413021F9145
:100320000F9108950F931F9305EA11E0C80140E86B
:1003300055E260E070E00E94C303C8010E94A4047B
:100340008DE061E00E94A7028EE060E00E94A702BB
:100350008FE060E00E94A70280E160E00E94A702B7
:1003600081E160E00E94A70282E160E00E94A702B2
:1003700083E160E00E94A70286E060E00E94A7029D
:1003800087E060E00E94A7028DE060E00E94A70283
:100390001F910F9108951F920F920FB60F92112483
:1003A0002F933F938F939F93AF93BF9380911801A7
:1003B00090911901A0911A01B0911B0130911C017B
:1003C0000196A11DB11D232F2D5F2D3720F02D5734
:1003D0000196A11DB11D20931C01809318019093DB
:1003E0001901A0931A01B0931B01809114019091FF
:1003F0001501A0911601B09117010196A11DB11D23
:100400008093140190931501A0931601B0931701E6
:10041000BF91AF919F918F913F912F910F900FBE00
:100420000F901F9018959B01AC017FB7F8948091B5
:10043000140190911501A0911601B091170166B5B4
:10044000A89B05C06F3F19F00196A11DB11D7FBF8C
:10045000BA2FA92F982F8827860F911DA11DB11D96
:1004600062E0880F991FAA1FBB1F6A95D1F7BC01D4
:100470002DC0FFB7F8948091140190911501A091BF
:100480001601B0911701E6B5A89B05C0EF3F19F022
:100490000196A11DB11DFFBFBA2FA92F982F882744
:1004A0008E0F911DA11DB11DE2E0880F991FAA1F9B
:1004B000BB1FEA95D1F7861B970B885E9340C8F265
:1004C000215030404040504068517C4F211531054B
:1004D0004105510571F60895789484B5826084BD14
:1004E00084B5816084BD85B5826085BD85B5816038
:1004F00085BDEEE6F0E0808181608083E1E8F0E098
:100500001082808182608083808181608083E0E8C6
:10051000F0E0808181608083E1EBF0E080818460A5
:100520008083E0EBF0E0808181608083EAE7F0E0A7
:10053000808184608083808182608083808181600B
:1005400080838081806880831092C1000895CF935A
:10055000DF93482F50E0CA0186569F4FFC0134912B
:100560004A575F4FFA018491882369F190E0880F20
:10057000991FFC01E859FF4FA591B491FC01EE5879
:10058000FF4FC591D491662351F42FB7F8948C9105
:10059000932F909589238C93888189230BC0623097
:1005A00061F42FB7F8948C91932F909589238C93B5
:1005B0008881832B88832FBF06C09FB7F8948C91C6
:1005C000832B8C939FBFDF91CF910895682F70E0AC
:1005D000CB0182559F4FFC012491CB0186569F4F42
:1005E000FC0144916A577F4FFB019491992319F4C0
:1005F00020E030E03CC0222351F1233071F0243060
:1006000028F42130A1F0223011F514C02630B1F0C9
:100610002730C1F02430D9F404C0809180008F7756
:1006200003C0809180008F7D8093800010C084B5CE
:100630008F7702C084B58F7D84BD09C08091B000E2
:100640008F7703C08091B0008F7D8093B000892F99
:1006500090E0880F991F84589F4FFC01A591B49199
:100660008C9120E030E0842311F021E030E0C901DA
:10067000089508951F920F920FB60F9211242F9391
:100680003F934F938F939F93EF93FF938091C0007D
:1006900082FD1DC04091C60020915D0130915E0138
:1006A0002F5F3F4F2F73307080915F0190916001F9
:1006B0002817390771F0E0915D01F0915E01E35E6A
:1006C000FE4F408330935E0120935D0102C0809114
:1006D000C600FF91EF919F918F914F913F912F9184
:1006E0000F900FBE0F901F901895E091B101F091FF
:1006F000B201E05CFF4F8191919120813181821B99
:10070000930B8F739070892B11F00E943903089519
:100710001F920F920FB60F9211242F933F938F9336
:100720009F93EF93FF932091A1013091A2018091BB
:10073000A3019091A4012817390731F48091C100D9
:100740008F7D8093C10014C0E091A301F091A401BA
:10075000EF59FE4F20818091A3019091A401019651
:100760008F7390709093A4018093A3012093C6008F
:10077000FF91EF919F918F913F912F910F900FBE1D
:100780000F901F901895AF92BF92DF92EF92FF9259
:100790000F931F93CF93DF93EC017A018B01DD243C
:1007A000403081EE580780E0680780E0780711F05C
:1007B000DD24D39491E0A92EB12CEC89FD89DD20B4
:1007C00069F0C50108A002C0880F991F0A94E2F7DA
:1007D000808360E079E08DE390E005C0108260E8FE
:1007E00074E88EE190E0A80197010E94E205215093
:1007F000304040405040569547953795279580E1C9
:100800002030380720F0DD2011F0DD24D6CFE88934
:10081000F9893083EA89FB89208319A2EE89FF894F
:10082000408121E030E0C9010C8C02C0880F991F83
:100830000A94E2F7482B4083EE89FF894081C90181
:100840000D8C02C0880F991F0A94E2F7482B408351
:10085000EE89FF894081C9010E8C02C0880F991F63
:100860000A94E2F7482B4083EE89FF8980810F8C40
:1008700002C0220F331F0A94E2F720952823208319
:10088000DF91CF911F910F91FF90EF90DF90BF907C
:10089000AF900895DC011C96ED91FC911D97E05CF2
:1008A000FF4F2191319180819181281B390B2F734A
:1008B0003070C9010895DC011C96ED91FC911D97E3
:1008C000E05CFF4F20813181E054F040DF01AE5BFE
:1008D000BF4F8D919C9111972817390719F42FEF6D
:1008E0003FEF07C08D919C91E80FF91F8081282F61
:1008F00030E0C9010895DC011C96ED91FC911D9733
:10090000E05CFF4F20813181E054F040DF01AE5BBD
:10091000BF4F8D919C9111972817390719F42FEF2C
:100920003FEF10C08D919C911197E80FF91F208126
:100930008D919C91119701968F73907011969C9355
:100940008E9330E0C9010895DC0191968C919197C6
:10095000882339F05496ED91FC915597808186FF5C
:10096000F9CF91961C920895CF93DF93EC01EE8519
:10097000FF85E05CFF4F20813181E054F0402F5F24
:100980003F4F2F733070DF01AE5BBF4F8D919C9155
:10099000119728173907D1F3E05CFF4F80819181CF
:1009A000E054F040E80FF91F6083EE85FF85E05CBE
:1009B000FF4F31832083EE89FF89208181E090E021
:1009C0000F8C02C0880F991F0A94E2F7282B20830E
:1009D00081E089A3EC89FD8980818064808381E046
:1009E00090E0DF91CF9108951092A8011092A70195
:1009F00088EE93E0A0E0B0E08093A9019093AA0173
:100A0000A093AB01B093AC0188E091E09093A60174
:100A10008093A5018DE191E09093B2018093B101A3
:100A200081E691E09093B4018093B30185EC90E06E
:100A30009093B6018093B50184EC90E09093B80157
:100A40008093B70180EC90E09093BA018093B90154
:100A500081EC90E09093BC018093BB0182EC90E02C
:100A60009093BE018093BD0186EC90E09093C0010D
:100A70008093BF0184E08093C10183E08093C20131
:100A800087E08093C30185E08093C40181E0809377
:100A9000C5010895CF93DF930E946C020E949201DA
:100AA000C5E7D3E00E9458012097E1F30E94750347
:100AB000F9CFCF92DF92EF92FF920F931F93CF93D4
:100AC000DF937C016B018A01C0E0D0E00FC0D6014A
:100AD0006D916D01D701ED91FC910190F081E02DB8
:100AE000C7010995C80FD91F015010400115110504
:100AF00071F7CE01DF91CF911F910F91FF90EF9091
:100B0000DF90CF900895EF92FF920F931F937B0198
:100B10008C01611571058105910529F420E030E013
:100B200040E050E00BC00E94DF00A80197010E9446
:100B30000406AC01CB01DA019C01AD01B901CA0187
:100B40001F910F91FF90EF900895EF92FF920F93F6
:100B50001F937B018C01621773078407950764F468
:100B6000261B370B480B590BCA01B9010E9483059C
:100B7000E60EF71E081F191FB701C8011F910F913C
:100B8000FF90EF900895629FD001739FF001829FC4
:100B9000E00DF11D649FE00DF11D929FF00D839F0C
:100BA000F00D749FF00D659FF00D9927729FB00DA9
:100BB000E11DF91F639FB00DE11DF91FBD01CF01BC
:100BC00011240895A1E21A2EAA1BBB1BFD010DC022
:100BD000AA1FBB1FEE1FFF1FA217B307E407F507ED
:100BE00020F0A21BB30BE40BF50B661F771F881FC9
:100BF000991F1A9469F760957095809590959B015F
:100C0000AC01BD01CF01089597FB092E05260ED03A
:100C100057FD04D0D7DF0AD0001C38F4509540951A
:100C2000309521953F4F4F4F5F4F0895F6F79095C0
:100C30008095709561957F4F8F4F9F4F0895EE0F70
:100C4000FF1F0590F491E02D09942F923F924F924F
:100C50005F926F927F928F929F92AF92BF92CF924C
:100C6000DF92EF92FF920F931F93CF93DF93CDB755
:100C7000DEB7CA1BDB0B0FB6F894DEBF0FBECDBFCD
:100C800009942A88398848885F846E847D848C849E
:100C90009B84AA84B984C884DF80EE80FD800C81A7
:100CA0001B81AA81B981CE0FD11D0FB6F894DEBF8A
:0C0CB0000FBECDBFED010895F894FFCFFA
:100CBC000100000000000000B40459054A047B0444
:040CCC005B04A4041D
:00000001FF
